:020000040000FA
:020000003BD1F2
:020008002ED1F7
:08001800D8CF01F0E8CF00F0A1
:10002000E0CF02F0EACF03F0E9CF04F09EAA02D0BD
:0E0030009DBA14D09EA802D09DB80AD0FF0041
:1000500050A202D09D98FCD081D8AD6EABB207D033
:10006000ABB40AD050B40ED0AE505BD8F1D0AB9840
:10007000AB88FA0E36D8ECD0AE50AB98AB88FB0EFE
:1000800030D8E6D0AE500B80FB0E2BD8E1D006C0A6
:10009000E9FF05C0EAFF1100C00E94124F0EAF6ECB
:1000A000240EAC6E900EAB6E506A09D811D8300E8B
:1000B0009D6E000E9F6ED08EC00EF26E1200000E6E
:1000C000546E566E5C0E556E576E509050821200F4
:1000D000000E586E5A6E6C0E596E5B6E50945086C0
:1000E00012009D9850B01BD056C0EAFF57C0E9FFE0
:1000F000EE6E000EEA6205D06C0EE96202D000EEF0
:100100005CF0EACF56F0E9CF57F05450566204D075
:100110005550576201D0508050929D8812009D88A2
:10012000120050B41AD05AC0EAFF5BC0E9FFEE6E6D
:10013000000EEA6205D07C0EE96202D000EE6CF09F
:10014000EACF5AF0E9CF5BF058505A6204D05950C8
:100150005B6201D0508450961200120050B21CD045
:1001600054C0EAFF55C0E9FFEECF53F0000EEA623B
:1001700005D06C0EE96202D000EE5CF0EACF54F0DC
:10018000E9CF55F05650546204D05750556201D013
:100190005082509053501200000C9D9A50B61DD0C2
:1001A00058C0EAFF59C0E9FFEECF52F0000EEA62F4
:1001B00005D07C0EE96202D000EE6CF0EACF58F078
:1001C000E9CF59F05A50586204D05B50596201D0BF
:1001D0005086509452509D8A12009D8A000C50B651
:1001E0001200DBDF7EDFFBD7120050B61200D5DF36
:1001F000106E105010AE0BD0116E146A11AC04D0FA
:1002000011AA010E156E1200020E156E1200146670
:1002100001D004D010C013F0146A08D010C012F03E
:10022000142A1450155C01E012001200900E115CAB
:1002300007E0800E115C05E0B00E115C03E01200D7
:06024000C5D0ECD0EDD0AA
:1002500004C0E9FF03C0EAFF02C0E0FF00C0E8FFFE
:1002600001C0D8FF1000EACF05F0E9CF06F0A1A247
:1002700002D0A0B229D0FF00896A8A6A8B6A926A8A
:10028000936A800E946E070EC16EC26A096A0A6A8A
:100290000B6A8B9C0768FF0EE82E4CEF01F0072ECF
:1002A0004BEF01F08B8CF40EF26FF36F00EE00F069
:1002B00010EE00F0F1DE03D8F5EC00F0FDD7010EF2
:1002C000B16EA282A0821200A192500EB26EB368EB
:1002D0000950896E0A508A6E0B508B6EF251F35D95
:1002E00014E0F2C0E9FFEA6A030EF22702E1F40E1D
:1002F000F26FEF5080EC02F0EE50100FE826E16E46
:10030000E26AEE50E66EEE50E66E210604E220064A
:1003100002E221680994230604E2220602E223682D
:100320000992250604E2240602E2256809902706C0
:1003300004E2260602E227680996290604E2280656
:1003400002E2296809982B0604E22A0602E22B68D9
:10035000099A2D0604E22C0602E22D680A9E2F0659
:1003600004E22E0602E22F680A9C310604E23006FF
:1003700002E231680A9A330604E2320602E2336886
:100380000A98350604E2340602E235680A96370612
:1003900004E2360602E237680A94390604E23806B7
:1003A00002E239680A923B0604E23A0602E23B683E
:1003B0000A903D0604E23C0602E23D680B9A3F06C5
:1003C00004E23E0602E23F680B9861D6135026E035
:1003D000135024E00F0EF76E12C0F6FF0800F55020
:1003E0001CE0F504086EEA6AF3C0E9FF0850EE6EFF
:1003F00013501324F66E0850100FF76E0900F5CF56
:1004000007F00900F550EE6E0750EE6EE95002E07D
:10041000F36F1200F40EF36F1200120012001200BC
:100420007B0E125C01E01200096A0A6A0B6A896A93
:060430008A6A8B6A1200CB
:10050000040DF950F350F9260984120009821200F3
:10051000098012000986120009881200098A120057
:100520000A8E12000A8C12000A8A12000A8812002F
:100530000A8612000A8412000A8212000A8012003F
:080540000B8A12000B88120067
:100F000000000000000000000000000000000000E1
:100F100000000000000000000000000000000000D1
:100F200000000000000000000000000000000000C1
:100F300000000000000000000000000000000000B1
:100F40000000000000000000010002030405060785
:100F50000008090A0B000C0D0E0F00100000000025
:100F60000000000000000000000000000000000081
:100F70000000000000000000000000000000000071
:10100000000032003E004A00560062006E007B0085
:10101000870093009F00AB00B700C300D000DC0046
:10102000E800F40000010C011801250131013D0127
:101030004901550161016D017A01860192019E010C
:10104000AA01B601C201CF01DB01E701F301FF01F3
:101050000B021702240230023C02480254026002D2
:101060006C027902850291029D02A902B502C102B9
:10107000CE02DA02E602F202FE020A03160323039C
:101080002F033B03470353035F036B03780384037E
:1010900090039C03A803B403C003CD03D903E50365
:1010A000F103FD030904150422042E043A04460446
:1010B00052045E046A04770483048F049B04A7042B
:1010C000B304BF04CC04D804E404F004FC04080511
:1010D000140521052D053905450551055D056905F1
:1010E000760582058E059A05A605B205BE05CB05D7
:1010F000D705E305EF05FB050706130620062C06BA
:10110000000032003E004A00560062006E007B0084
:10111000870093009F00AB00B700C300D000DC0045
:10112000E800F40000010C011801250131013D0126
:101130004901550161016D017A01860192019E010B
:10114000AA01B601C201CF01DB01E701F301FF01F2
:101150000B021702240230023C02480254026002D1
:101160006C027902850291029D02A902B502C102B8
:10117000CE02DA02E602F202FE020A03160323039B
:101180002F033B03470353035F036B03780384037D
:1011900090039C03A803B403C003CD03D903E50364
:1011A000F103FD030904150422042E043A04460445
:1011B00052045E046A04770483048F049B04A7042A
:1011C000B304BF04CC04D804E404F004FC04080510
:1011D000140521052D053905450551055D056905F0
:1011E000760582058E059A05A605B205BE05CB05D6
:1011F000D705E305EF05FB050706130620062C06B9
:10120000000032003E004A00560062006E007B0083
:10121000870093009F00AB00B700C300D000DC0044
:10122000E800F40000010C011801250131013D0125
:101230004901550161016D017A01860192019E010A
:10124000AA01B601C201CF01DB01E701F301FF01F1
:101250000B021702240230023C02480254026002D0
:101260006C027902850291029D02A902B502C102B7
:10127000CE02DA02E602F202FE020A03160323039A
:101280002F033B03470353035F036B03780384037C
:1012900090039C03A803B403C003CD03D903E50363
:1012A000F103FD030904150422042E043A04460444
:1012B00052045E046A04770483048F049B04A70429
:1012C000B304BF04CC04D804E404F004FC0408050F
:1012D000140521052D053905450551055D056905EF
:1012E000760582058E059A05A605B205BE05CB05D5
:1012F000D705E305EF05FB050706130620062C06B8
:10130000000032003E004A00560062006E007B0082
:10131000870093009F00AB00B700C300D000DC0043
:10132000E800F40000010C011801250131013D0124
:101330004901550161016D017A01860192019E0109
:10134000AA01B601C201CF01DB01E701F301FF01F0
:101350000B021702240230023C02480254026002CF
:101360006C027902850291029D02A902B502C102B6
:10137000CE02DA02E602F202FE020A031603230399
:101380002F033B03470353035F036B03780384037B
:1013900090039C03A803B403C003CD03D903E50362
:1013A000F103FD030904150422042E043A04460443
:1013B00052045E046A04770483048F049B04A70428
:1013C000B304BF04CC04D804E404F004FC0408050E
:1013D000140521052D053905450551055D056905EE
:1013E000760582058E059A05A605B205BE05CB05D4
:1013F000D705E305EF05FB050706130620062C06B7
:10140000000032003E004A00560062006E007B0081
:10141000870093009F00AB00B700C300D000DC0042
:10142000E800F40000010C011801250131013D0123
:101430004901550161016D017A01860192019E0108
:10144000AA01B601C201CF01DB01E701F301FF01EF
:101450000B021702240230023C02480254026002CE
:101460006C027902850291029D02A902B502C102B5
:10147000CE02DA02E602F202FE020A031603230398
:101480002F033B03470353035F036B03780384037A
:1014900090039C03A803B403C003CD03D903E50361
:1014A000F103FD030904150422042E043A04460442
:1014B00052045E046A04770483048F049B04A70427
:1014C000B304BF04CC04D804E404F004FC0408050D
:1014D000140521052D053905450551055D056905ED
:1014E000760582058E059A05A605B205BE05CB05D3
:1014F000D705E305EF05FB050706130620062C06B6
:10150000000032003E004A00560062006E007B0080
:10151000870093009F00AB00B700C300D000DC0041
:10152000E800F40000010C011801250131013D0122
:101530004901550161016D017A01860192019E0107
:10154000AA01B601C201CF01DB01E701F301FF01EE
:101550000B021702240230023C02480254026002CD
:101560006C027902850291029D02A902B502C102B4
:10157000CE02DA02E602F202FE020A031603230397
:101580002F033B03470353035F036B037803840379
:1015900090039C03A803B403C003CD03D903E50360
:1015A000F103FD030904150422042E043A04460441
:1015B00052045E046A04770483048F049B04A70426
:1015C000B304BF04CC04D804E404F004FC0408050C
:1015D000140521052D053905450551055D056905EC
:1015E000760582058E059A05A605B205BE05CB05D2
:1015F000D705E305EF05FB050706130620062C06B5
:10160000000032003E004A00560062006E007B007F
:10161000870093009F00AB00B700C300D000DC0040
:10162000E800F40000010C011801250131013D0121
:101630004901550161016D017A01860192019E0106
:10164000AA01B601C201CF01DB01E701F301FF01ED
:101650000B021702240230023C02480254026002CC
:101660006C027902850291029D02A902B502C102B3
:10167000CE02DA02E602F202FE020A031603230396
:101680002F033B03470353035F036B037803840378
:1016900090039C03A803B403C003CD03D903E5035F
:1016A000F103FD030904150422042E043A04460440
:1016B00052045E046A04770483048F049B04A70425
:1016C000B304BF04CC04D804E404F004FC0408050B
:1016D000140521052D053905450551055D056905EB
:1016E000760582058E059A05A605B205BE05CB05D1
:1016F000D705E305EF05FB050706130620062C06B4
:10170000000032003E004A00560062006E007B007E
:10171000870093009F00AB00B700C300D000DC003F
:10172000E800F40000010C011801250131013D0120
:101730004901550161016D017A01860192019E0105
:10174000AA01B601C201CF01DB01E701F301FF01EC
:101750000B021702240230023C02480254026002CB
:101760006C027902850291029D02A902B502C102B2
:10177000CE02DA02E602F202FE020A031603230395
:101780002F033B03470353035F036B037803840377
:1017900090039C03A803B403C003CD03D903E5035E
:1017A000F103FD030904150422042E043A0446043F
:1017B00052045E046A04770483048F049B04A70424
:1017C000B304BF04CC04D804E404F004FC0408050A
:1017D000140521052D053905450551055D056905EA
:1017E000760582058E059A05A605B205BE05CB05D0
:1017F000D705E305EF05FB050706130620062C06B3
:10180000000032003E004A00560062006E007B007D
:10181000870093009F00AB00B700C300D000DC003E
:10182000E800F40000010C011801250131013D011F
:101830004901550161016D017A01860192019E0104
:10184000AA01B601C201CF01DB01E701F301FF01EB
:101850000B021702240230023C02480254026002CA
:101860006C027902850291029D02A902B502C102B1
:10187000CE02DA02E602F202FE020A031603230394
:101880002F033B03470353035F036B037803840376
:1018900090039C03A803B403C003CD03D903E5035D
:1018A000F103FD030904150422042E043A0446043E
:1018B00052045E046A04770483048F049B04A70423
:1018C000B304BF04CC04D804E404F004FC04080509
:1018D000140521052D053905450551055D056905E9
:1018E000760582058E059A05A605B205BE05CB05CF
:1018F000D705E305EF05FB050706130620062C06B2
:10190000000032003E004A00560062006E007B007C
:10191000870093009F00AB00B700C300D000DC003D
:10192000E800F40000010C011801250131013D011E
:101930004901550161016D017A01860192019E0103
:10194000AA01B601C201CF01DB01E701F301FF01EA
:101950000B021702240230023C02480254026002C9
:101960006C027902850291029D02A902B502C102B0
:10197000CE02DA02E602F202FE020A031603230393
:101980002F033B03470353035F036B037803840375
:1019900090039C03A803B403C003CD03D903E5035C
:1019A000F103FD030904150422042E043A0446043D
:1019B00052045E046A04770483048F049B04A70422
:1019C000B304BF04CC04D804E404F004FC04080508
:1019D000140521052D053905450551055D056905E8
:1019E000760582058E059A05A605B205BE05CB05CE
:1019F000D705E305EF05FB050706130620062C06B1
:101A0000000032003E004A00560062006E007B007B
:101A1000870093009F00AB00B700C300D000DC003C
:101A2000E800F40000010C011801250131013D011D
:101A30004901550161016D017A01860192019E0102
:101A4000AA01B601C201CF01DB01E701F301FF01E9
:101A50000B021702240230023C02480254026002C8
:101A60006C027902850291029D02A902B502C102AF
:101A7000CE02DA02E602F202FE020A031603230392
:101A80002F033B03470353035F036B037803840374
:101A900090039C03A803B403C003CD03D903E5035B
:101AA000F103FD030904150422042E043A0446043C
:101AB00052045E046A04770483048F049B04A70421
:101AC000B304BF04CC04D804E404F004FC04080507
:101AD000140521052D053905450551055D056905E7
:101AE000760582058E059A05A605B205BE05CB05CD
:101AF000D705E305EF05FB050706130620062C06B0
:101B0000000032003E004A00560062006E007B007A
:101B1000870093009F00AB00B700C300D000DC003B
:101B2000E800F40000010C011801250131013D011C
:101B30004901550161016D017A01860192019E0101
:101B4000AA01B601C201CF01DB01E701F301FF01E8
:101B50000B021702240230023C02480254026002C7
:101B60006C027902850291029D02A902B502C102AE
:101B7000CE02DA02E602F202FE020A031603230391
:101B80002F033B03470353035F036B037803840373
:101B900090039C03A803B403C003CD03D903E5035A
:101BA000F103FD030904150422042E043A0446043B
:101BB00052045E046A04770483048F049B04A70420
:101BC000B304BF04CC04D804E404F004FC04080506
:101BD000140521052D053905450551055D056905E6
:101BE000760582058E059A05A605B205BE05CB05CC
:101BF000D705E305EF05FB050706130620062C06AF
:101C0000000032003E004A00560062006E007B0079
:101C1000870093009F00AB00B700C300D000DC003A
:101C2000E800F40000010C011801250131013D011B
:101C30004901550161016D017A01860192019E0100
:101C4000AA01B601C201CF01DB01E701F301FF01E7
:101C50000B021702240230023C02480254026002C6
:101C60006C027902850291029D02A902B502C102AD
:101C7000CE02DA02E602F202FE020A031603230390
:101C80002F033B03470353035F036B037803840372
:101C900090039C03A803B403C003CD03D903E50359
:101CA000F103FD030904150422042E043A0446043A
:101CB00052045E046A04770483048F049B04A7041F
:101CC000B304BF04CC04D804E404F004FC04080505
:101CD000140521052D053905450551055D056905E5
:101CE000760582058E059A05A605B205BE05CB05CB
:101CF000D705E305EF05FB050706130620062C06AE
:101D0000000032003E004A00560062006E007B0078
:101D1000870093009F00AB00B700C300D000DC0039
:101D2000E800F40000010C011801250131013D011A
:101D30004901550161016D017A01860192019E01FF
:101D4000AA01B601C201CF01DB01E701F301FF01E6
:101D50000B021702240230023C02480254026002C5
:101D60006C027902850291029D02A902B502C102AC
:101D7000CE02DA02E602F202FE020A03160323038F
:101D80002F033B03470353035F036B037803840371
:101D900090039C03A803B403C003CD03D903E50358
:101DA000F103FD030904150422042E043A04460439
:101DB00052045E046A04770483048F049B04A7041E
:101DC000B304BF04CC04D804E404F004FC04080504
:101DD000140521052D053905450551055D056905E4
:101DE000760582058E059A05A605B205BE05CB05CA
:101DF000D705E305EF05FB050706130620062C06AD
:101E0000000032003E004A00560062006E007B0077
:101E1000870093009F00AB00B700C300D000DC0038
:101E2000E800F40000010C011801250131013D0119
:101E30004901550161016D017A01860192019E01FE
:101E4000AA01B601C201CF01DB01E701F301FF01E5
:101E50000B021702240230023C02480254026002C4
:101E60006C027902850291029D02A902B502C102AB
:101E7000CE02DA02E602F202FE020A03160323038E
:101E80002F033B03470353035F036B037803840370
:101E900090039C03A803B403C003CD03D903E50357
:101EA000F103FD030904150422042E043A04460438
:101EB00052045E046A04770483048F049B04A7041D
:101EC000B304BF04CC04D804E404F004FC04080503
:101ED000140521052D053905450551055D056905E3
:101EE000760582058E059A05A605B205BE05CB05C9
:101EF000D705E305EF05FB050706130620062C06AC
:101F0000000032003E004A00560062006E007B0076
:101F1000870093009F00AB00B700C300D000DC0037
:101F2000E800F40000010C011801250131013D0118
:101F30004901550161016D017A01860192019E01FD
:101F4000AA01B601C201CF01DB01E701F301FF01E4
:101F50000B021702240230023C02480254026002C3
:101F60006C027902850291029D02A902B502C102AA
:101F7000CE02DA02E602F202FE020A03160323038D
:101F80002F033B03470353035F036B03780384036F
:101F900090039C03A803B403C003CD03D903E50356
:101FA000F103FD030904150422042E043A04460437
:101FB00052045E046A04770483048F049B04A7041C
:101FC000B304BF04CC04D804E404F004FC04080502
:101FD000140521052D053905450551055D056905E2
:101FE000760582058E059A05A605B205BE05CB05C8
:101FF000D705E305EF05FB050706130620062C06AB
:020000040030CA
:0E000000FFFEFEFEFFFEFAFFFFFFFFFFFFFF09
:00000001FF
